:020000020000FC
:02000000EDC051
:04000C0060C002C00E
:100014000F930FB70F931F93EF93FF930CB11BB183
:100024001871112309F02CC050FD01C011C00D93AB
:10003400019731F55E7F82E390E0A2E9B0E0C0E68B
:10004400D0E00D9109930197E1F70AEAA2D018C014
:1000540000951FE0101BA0F0E2E3F0E0E10F09942B
:1000640017C01AC01EC021C024C011C010C00FC0C8
:100074000EC00DC00CC00BC00AC009C008C01DC012
:10008400FF91EF911F910F910FBF0F911895F8CF2A
:1000940050680AEA7ED0F4CF5F77F8948AD039D0DA
:1000A400ADCFEEE0F2E079D0EBCFE0E2F2E075D054
:1000B400E7CFEAE2F2E071D0E3CF38EC949882E340
:1000C40090E0A2E9B0E05160DBCF0F930FB70F933C
:1000D4001F933A9541F402B310E1012702BB38ECB7
:1000E40050FD01C08BCF2A95213011F4929A08C09B
:1000F400222331F4002703BF57FD0BD025E092984B
:100104000CED02BF05E003BF1F910F910FBF0F91CC
:100114001895BF93AF930F938F939F93939808ED84
:100124000A95F1F7939A0FE00A95F1F70F2D10D085
:10013400A0E6B0E082E390E00D910AD00197E1F7E8
:1001440005E527D09F918F910F91AF91BF910895AD
:10015400889415D0079513D0079511D007950FD023
:1001640007950DD007950BD0079509D0079507D0B3
:10017400079505D0089403D0089401D0089516E09B
:1001840020F4939A1A95F1F7089593981A95F1F734
:1001940008955D9BFECF0CB90895EF93FF93C89526
:1001A400002D3196F6DF002009F0F9CFFF91EF9191
:1001B4000895FF93EF938F939F930F93E0E6F0E0FE
:1001C40084E690E0002701930197E9F70F919F914E
:1001D4008F91EF91FF910895F8940FED0DBF55277E
:1001E400FF2438ECE6DF0CE101BB08E102BB02E0CE
:1001F40009BF0CED02BF05E003BF25E003E009B928
:10020400579A539A549A7894FFCF3233322D444DEF
:10021400582035302056312E3120200032383131EB
:0A0224003034303300003035300074
:00000001FF
